:030000000219FDE5
:03000B000200AA46
:03002B0002015679
:03005B000202E8B6
:030073000202D5B1
:1000800002030406080C10182030406080040608A3
:100090000C10182030406080A0C00003070F1F0D17
:1000A0000D0403060D0502030202C2AFC0D0C0E07A
:1000B000206214E5256009E473E525F4F58AD2622F
:1000C000D0E0D0D0D2AF3285268AC262E526F46075
:1000D00029D0E0D0D0C293C295C297D2AF32C2939A
:1000E000C295C297206F0C206509740ED5E0FDE51E
:1000F0007B4290D0E0D0D0D2AF32758A00C28DD290
:100100006201F301B9306805206502D29301B9306C
:100110006805206502D29501B9306805206502D2D4
:100120009701B9C29230680A206507740CD5E0FDCA
:10013000D29301B9C29430680A206507740CD5E0E7
:10014000FDD29501B9C29630680A206507740CD5B6
:10015000E0FDD29701B9C2AFC2AD53E6EFC0D0C047
:10016000E0D2D3D2AFC2CEE52A600720744F152A61
:1001700021BD7800790020742EE580307E01F430B6
:10018000E30278FF53DACF207E0343DA20307E0388
:1001900043DA10C2D8C271E580307E01F430E30248
:1001A00079FFC3E89970CB306103752A402074034E
:1001B000752A40885CD270E86003755F0020740D7A
:1001C000E52B6004152B21CD43DA01C2D820700243
:1001D00021E0A85C206102C27020740221DE882226
:1001E0007882B6040385222420CF0AD0E0D0D04301
:1001F000E610D2AD32C2CF053A7802E52A6005306A
:100200007402152AC3E55C94014005755F00412125
:10021000756000756900E55F2401F55F5003755F47
:10022000FF7982B7020D306E1DC3E522943240166D
:10023000854C227982B7030E306E0BC3E5229432CF
:100240004004798E8722C3E5239522600840041577
:100250002341550523D8CA0569E56970021569D59A
:100260006A69756A017808E56B60497805C3E569D4
:10027000956B4057C3E569956C50087801756A0322
:1002800002028FC3E569956D50057801756A01C357
:10029000E5629524401E7982B7040241C0206E14A5
:1002A000852462E569046003856B69756A017523BD
:1002B0003C0202CBE5622850057562FF41C0F56241
:1002C000E5620470067560FF7569FFD0E0D0D04329
:1002D000E610D2AD32C2AF53E67F7592FA7593FF46
:1002E000C260759104D2AF32C2AF53E6EFC2ADC067
:1002F000D0C0E0C0F0D2D3D2AFA8FBA9FCC2D830A6
:100300007102614F53DACF207E0343DA10307E034F
:1003100043DA20D271E580307E01F420E3026126C9
:1003200088278928A13453DACF207E0343DA20308E
:100330007E0343DA10C2D8C271307402A120780063
:10034000E580307E01F430E302A120885CA10853EF
:10035000DACF207E0343DA20307E0343DA10C27105
:10036000206102812853DACF207E0343DA10307EE9
:100370000343DA20C2D8D27188578958C3E895550B
:10038000F8E99556F97B007E087A00C3E8948CE979
:1003900094005005755B00811A882178A2E6A82197
:1003A0006055C3E894C8E994005008E4D2E4FB7AAD
:1003B0000A61F5C3E89468E994015008E4D2E3FBCC
:1003C0007A0F61F5C3E894D0E994025008E4D2E2D0
:1003D000FB7A1E61F5C3E894A0E994055008E4D2C5
:1003E000E1FB7A3C61F5C3E89498E994085008E48D
:1003F000D2E0FB7A787E00C3E89559FCE9955AFD76
:1004000030E70AECF42401FCEDF43400FD755B00E8
:10041000C3EC9AED9E5003755B018859895A855744
:10042000558558567802A108C3E89527F8E995281C
:10043000F9307C0281EC307B0281EC307A0281E57C
:10044000207502814BE9FDE8FC816AE9C313F9E8F4
:1004500013F830790281E5E9C313F9E813F830782D
:100460000281E5E9C313FDE813FC20612CC3EC9481
:0F0470001CED940240028181ED701EC3EC94C814
:10047F0050180529E52970021529C3E529940A505A
:10048F0002A120755C00D270A120E5296002152918
:10049F007400207F037896E624FAFEE43400FFC34D
:1004AF00EC9EFCED9FFD50067800790081ECC3ECCB
:1004BF0094FFED9400400678FF790081ECEC857293
:1004CF00F0A4C5F0A2F733F87900400302050878CD
:1004DF00FF7900020508E9C313F9E813F8307C0E21
:1004EF00E9600278FFC3E81338F8E43400F9C3E891
:1004FF0094FFE99400400278FF885CD2702061027B
:10050F00A120741FF4552F4BF52FC274EB7002D23C
:10051F0074752A40307403752A0A306102A13420A1
:10052F00740353DAFE207403752B20D0F0D0E0D083
:10053F00D0D2AD43E610327901020564790302058A
:10054F0064790A020564791E020564796402056400
:10055F0079C80205647817E4D5E0FDD8FAD9F622F8
:10056F007A147B7802058B7A107B8C02058B7A0DBF
:10057F007BB402058B7A0B7BC802058BE573D5E044
:10058F0001227902E4C294D5E0FDD295D5E0FDC2F7
:10059F0095D5E0FDD294D5E0FDE920E002D293306D
:1005AF00E002D297E573D5E0FDE920E002C2933077
:1005BF00E002C2977496D5E0FDD9C9EAF8D5E0FDFF
:1005CF00D8FBDBB8C29422C37C007D0075F0000518
:1005DF00F0EA33FAEB33FB50F6EB13FBEA13FAC3F3
:1005EF00E9FFE8FEE89AF8E99BF95004EFF9EEF815
:1005FF00B3EC33FCED33FDD5F0DFEDF9ECF822E889
:10060F0089F08A20D2D4F8A9F07B0030F70B7BFF5A
:10061F00F42401F8E9F43400F9E88520F0A4ADF0F2
:10062F00F8E98520F0A4AFF0FEED2EF974003FFA43
:10063F007C04C3EA13FAE913F9E813F8DCF48BF03E
:10064F0030F70AE8F42401F8E9F43400F9E889F006
:10065F00C2D4F8A9F0227882B60403020704C3E5D6
:10066F005C9419401EE52D54067018206E367805DF
:10067F007994E7146007780A1460027812C3E54191
:10068F0098401F306E098564627569FF756A018530
:10069F002224E4F544F545F546F547F548C26E02C8
:1006AF000704D26E7994E7147013E523F43333F90A
:1006BF0013F8E9540104F9E854FE0206F8E714149C
:1006CF007014E523F4333333F913F8E9540304F9C1
:1006DF00E854FC020700E523F433333333F913F8FE
:1006EF00E954070404F9E854F8C39440F8E9940076
:1006FF00F98844894522C3E54113F9E54013F8C34E
:10070F00E54498F8E54599F9500CC3E89480E994CD
:10071F00FF401602073CC3E8947FE99400500302A0
:10072F00073C787F790002073C788079FF884989F8
:10073F004A22E5492546F8E54A3547F9854A20E436
:10074F00300701F43548FA30E709C3EA94F0401551
:10075F0002077AC3EA940F500302077A78FF79FFF2
:10076F007A0F02077A780079007AF0C3E524956151
:10077F00500AC374019524500B020798E54A20E7ED
:10078F000E020798E54A30E706884689478A4822CD
:10079F0078A5E6FAC3E54933F8E54A33F9D10EE90E
:1007AF0030E70BC3E89480E994FF4013E1D2C3E82C
:1007BF00947FE994005002E1D2787F7900E1D278FA
:1007CF008079FFE820E715C3E52398F84009C3E8CF
:1007DF00940140030207F978010207F9E8F42401B4
:1007EF002523F840030207F978FF884B2278A6E605
:1007FF00FAA847A94812060EE930E70CC3E894019E
:10080F00E994FF401602082EC3E894FFE9940050C4
:10081F000302082E78FF790002082E780179FFE98C
:10082F0020E715C3E54B98F84009C3E8940140034E
:10083F000208557801020855E8F42401254BF840C9
:10084F000302085578FF88242278FF20692879A1B0
:10085F00E76023E541601F74FF8541F0848539F01F
:0F086F00306A0375F005A4F8C5F0600278FFC386
:10087E00E895645002A864886322C3E5409440E57D
:10088E00419401E5635003140199046002F563225B
:10089E007883E6F520120F3675E89012054675E856
:1008AE009030EDFDA8BDA9BE120FDD756E30756FCF
:1008BE0000C3740013FD7430606613FC74302CFC9E
:1008CE0074003DFDECFAEDFBC3E89AE99B4014E59C
:1008DE006E2430F56EE56F3400F56FEA2CFAEB3DC1
:1008EE00FB80E5AE6EAF6FC3E56F13F9E56E13F8DF
:1008FE00C3E913F9E813F87A03C3E913F9E813F817
:10090E00DAF7AA201A7009756E00756F0002092EAB
:10091E001AEA6008EE28FEEF39FFDAF88E6E8F6F56
:10092E002275E890227883E6FF30EDF9A8BDA9BEC6
:10093E000570C3E57094084052757000E9FA79A00D
:10094E00E76044EA7007E571601B020967C3E8952A
:10095E00716010E5715006600C140209730460F9A1
:10096E00020973E571F571C394A8401B7561C0C38C
:10097E0094054013756180C39405400B756140C3A7
:10098E009405400375610075BB0122EFC3940160AD
:10099E001F7430601BC3E894FFE994035012C3E840
:1009AE00956EE9956F5009E561600C15610209C5F8
:1009BE00E561F460020561A861C3E524985002A8C0
:1009CE0024C3E89562400AA862E562F4600385627A
:1009DE006188258826E570B4070375BB1E22743224
:1009EE0079A787F0A4C5F0A2F733F8C3E895614064
:1009FE0002A861882288248825882688642275406A
:100A0E00007541F022C2AF75C820A8CCA9CDAA3A74
:100A1E0030CF010A75C824D2AFAB3BAC3C883B89C2
:100A2E003CC3E89BF8E99C206908F9306602612412
:100A3E00417EAD3D8A3DF9EA9DFA600678FF79FF69
:100A4E004163AE3EAF3F8B3E8C3FA83BA93CC3E813
:100A5E009EF8E99FF9C3E54113FBE54013FAE82A36
:100A6E00F540E93BF54150067540FF7541FF41CB1E
:100A7E00AA40AB41AC40AD417E047F02C3EB94046F
:100A8E00400D1E1FC3EB94084005206A021E1FC3B3
:100A9E00ED13FDEC13FCDEF7C3EA9CFAEB9DFBEFC6
:100AAE006009C3E913F9E813F8DFF7EA28FAEB391E
:100ABE00FB8A408B4150067BFF8B408B41C3EB94EE
:100ACE00025002D2663069047F0341F67892E6FF47
:100ADE00C3E537948240110FC3E53794A040010F50
:100AEE00C3EF940640027F057E02E541C4540FF920
:100AFE00E541C454F0F8E540C4540F28F8C3E89E0D
:100B0E00FAE99400FB4009C3EA9402EB9400500406
:100B1E007A02E4FB6170AA40AB41EBC4FEEAC45416
:100B2E000F4EFCC3EA9CFAEB9400FBC3E813C3130D
:100B3E00F8EA28FAEB3400FB8A408B41C3EB9402AF
:100B4E004002C2667802EBC4FE7B00EAC4540F4E2C
:100B5E00FAC3EA98FA4005C3940250027A027892D8
:100B6E00E6FF3060026170855192855293D26043E8
:100B7E00E680C3E49AF8E49BF930660261FCE8FA79
:100B8E00E9FBD3E913FDE813FC88518952C3EF94B6
:100B9E00036038EF20E00DE82CF8E93DF9ECFAEDB2
:100BAE00FB020BC5E828F8E939F9C3E82402F8E995
:100BBE003400F97AFE7BFFC3EF9403400E8A538B09
:100BCE0054884D894E8C4F8D508130885389548A6C
:100BDE004D8B4E8C4F8D503069127553F07554FFFE
:100BEE00754FF07550FF7551F07552FF8130E8FA70
:100BFE00D3E813FC8851C3EF94036020EF20E00785
:100C0E00E82CF8ECFA811CE8282402F87AFEC3EFEF
:100C1E00940340088A53884D8C4F813088538A4DF7
:100C2E008C4FE568C3335002646BF5683060028107
:100C3E003A753402D26043E680E52D54066034A83E
:100C4E0040A941C3E913F9E813F8C3E913F9E8130E
:100C5E00F8306904E92440F9C2AF53E67F7591007C
:0E0C6E00C3E498F594E499F595759104D2606D
:100C7C0043E680D2AF22D264754300752000306CFD
:100C8C0003752040020CA1D26475430075204030DE
:100C9C006C0375200078017901206620E52D54063F
:100CAC006002C2647914E541C313700104F8C39463
:100CBC001440027814306904781B791B206010E50D
:100CCC0043600C306903D53404D26DA154914205B4
:100CDC0043E59E7005E59B020CE8E59A5440B5206F
:100CEC0002A13E30690908C3E89940011881C82067
:100CFC00640A08C3E899400281A181C8C264C2AFEA
:100D0C0053E67F7591003066127594007595F875F1
:100D1C009104D26043E680D2AF81A1E5417EFFC34E
:100D2C00334005C3334001FEC3E49E759400F59532
:100D3C00A11BC3E5339401500281A130640281A14F
:100D4C00D802A15281C8C26DC2AF53E67F75910023
:100D5C00855394855495759104854D92854E93D207
:100D6C006043E680D2AFE52D54066008206A020588
:100D7C0033020D90306D0D206C0A2064071581151F
:100D8C008102165E2278003064027801E53775F036
:100D9C0007A4F9E5F028F5F0E9A2F013A2F113A2EB
:100DAC00F213F537C394785003753778C3E537954C
:100DBC00384008D265C293C295C297306002A1C771
:100DCC00854F92855093D26043E68022207D19C2D4
:100DDC00AF754202C294D292306202D297D2AF75F2
:100DEC009F33759E00020FDAC2AF754202C294D2D5
:100DFC0096306202D293D2AF759F33759E00020F6C
:100E0C00DA307243207D20C2AF75420390013475F5
:100E1C007B10C297C296306204D295C12BD294D269
:100E2C00AF759E23020FDAC2AF7542039001347581
:100E3C007B10C293C292306204D295C14BD294D231
:100E4C00AF759E22020FDA207D17C2AF7542039058
:100E5C00010FC297306202D295D2AF759E23020F5A
:100E6C00DAC2AF75420390010FC293306202D29581
:100E7C00D2AF759E22020FDA207D16C2AF754204E6
:100E8C00C292D296306202D295D2AF759E22020FD8
:100E9C00DAC2AF754204C296D292306202D295D2B7
:100EAC00AF759E23020FDA307249207D23C2AF75D5
:100EBC004205900123757B04C295C294306204D222
:100ECC0093C1D1D292D2AF759F33759E00020FDAC7
:100EDC00C2AF754205900145757B40C295C29430F6
:100EEC006204D297C1F4D296D2AF759F33759E002F
:100EFC00020FDA207D1AC2AF754205900105C2952A
:100F0C00306202D293D2AF759F33759E00020FDA16
:100F1C00C2AF754205900119C2953062E8D297D2E2
:100F2C00AF759F33759E00020FDA207D16C2AF7528
:100F3C004206C296D294306202D293D2AF759E23EF
:100F4C00020FDAC2AF754206C292D294306202D25C
:100F5C0097D2AF759E22020FDA307244207D20C2E8
:100F6C00AF754201900145757B40C293C2923062CD
:100F7C0004D297E183D296D2AF759E22020FDAC2C9
:100F8C00AF754201900123757B04C297C296306203
:100F9C0005D293020FA4D292D2AF759E23020FDA20
:100FAC00207D17C2AF754201900119C293306202C5
:100FBC00D297D2AF759E22020FDAC2AF7542019062
:100FCC000105C297306202D293D2AF759E23C265DF
:100FDC0022900103757B00C293C295C297C292C244
:100FEC0094C296C26222788076070876070876014A
:100FFC000876040876FF0876FF087607087602085C
:10100C007601087601788C76010876000876B408AB
:10101C0076FF0876FF0876FF0876030876FF0876D9
:10102C00010876FF0876250876D00876780876C809
:10103C000876040876FF08760108760008767A08A8
:10104C0076100876010876010876000876FF087697
:10105C0000227887E6FFC2727888C27DE630E10212
:0E106C00D27DC27E7889E630E102D27EC3EFEB
:10107A0094026008758E01D27302108B758E00C2BD
:10108A0073227880E6149000809378A5F67881E63A
:10109A00149000809378A6F67886E61490008D93D3
:1010AA0078A7F6789FE6F87005756B0001D2C3E859
:1010BA00941140027811E82828F56B256B256B28D6
:1010CA00F56C256B2828F56D7886E6F539C3940208
:1010DA005003753902789CE67538FFB402037538F7
:1010EA00A0B4030375388278A3E61490009A93F5A6
:1010FA0066120FDD22227896E6FA7897E6FB788860
:10110A00E6B40305C3EB940EFB307F047A007BFF41
:10111A00C3EB9AFCC3948250027C827572000572FA
:10112A00EC8572F0A4C3E5F0947D40F222D27F31BF
:10113A00001205551205557A007B007C1012054BEA
:10114A00E55C2AFA74003BFBDCF37C04C3EB13FB7B
:10115A00EA13FADCF7FEC27F310022757C00757D46
:10116A0000E5EF20E6037520000520903DFFE5200D
:10117A00146006901FFF1460009304600375EF1655
:10118A0053D9BF7581C043FF8012054675EF0643E8
:10119A00B203E5B3240220E70DF521E5B120E0060C
:1011AA008521B343B101120FDD7580FF75A4007567
:1011BA00F1FE75D4F775900275A5FC75F2FC75D52C
:1011CA000075A0FD75A60275F30275D60075B0FF0D
:1011DA0075A70175F4FF75E241120FDDE4F8F6D840
:1011EA00FD756801120FF21216B57898867375307C
:1011FA0001C2AF12055F12056F120555120576126C
:10120A00055512057D1205551217E812055F1205DC
:10121A005F12055AC2AF757C00757D0078FA79FABB
:10122A00308307D9FBD8F7021C00115E118C11FF1D
:10123A00310078988673120FDD75881075890275EA
:10124A00C82475910475D84075A82275B80275E648
:10125A0090759B80759D00759A80759C0075D10E5E
:10126A0075BC5875BB0175BA1F75E880120546D260
:10127A00AF12089E75360053DACF207E0343DA2078
:10128A00307E0343DA1043DA01C2D8C27112055F15
:10129A00D2617B037A0CE55B70077A0CDB030212DE
:1012AA001E12055520700302121EC270E55CC3941B
:1012BA000240E1E52F541F855E5DF55EB55DD5DA26
:1012CA00D5C26153DACF207E0343DA20307E03434E
:1012DA00DA10C2D8C27178A2E67008D274E52F5427
:1012EA00E0F52FC27575290012055A307409C3E555
:1012FA0029940A4002D27512054B7802307402789A
:10130A0000C3E55C9840F0C2AF12056F12056F1278
:10131A00056FD2AF12055F754C0012054B788CE64B
:10132A00C394015003021411E530C394015003021F
:10133A001411757CA5757DF1207435C3E55C94FFA5
:10134A005003021411C2AF120584D2AF12055AC358
:10135A00E55C940150EFC2AF12056F1205501205F9
:10136A006FD2AF12055AC3E55C94FF40E902186DCB
:10137A007F05D27F310012055AC2AFC27F3100AE5B
:10138A005CC3E55C947FD2AF50028121120546C24C
:10139A00AF120584D2AFDFDA3137C3EE94057897FE
:1013AA00F612055F1217F07F0AD27F310012055A32
:1013BA00C2AFC27F3100AE5CC3E55C947FD2AF504E
:1013CA00E6120546C2AF12056F12055012056FD21A
:1013DA00AFDFD63137EE24037896F6F87997E7C36C
:1013EA0094824003985006E824827897F612055FA3
:1013FA0012170312181F12055A3100C3E55C94FF35
:10140A005002613C02186D757C00757D00C3E55C75
:10141A00954C4003855C4C12055A78017988E7B4EB
:10142A0003027805C3E55C9840026124C2AF120545
:10143A0084120584120584D2AF12055F753000E468
:10144A00F531F5320531E531F4703F0532789AE627
:10145A007819146012783214600D787D1460087857
:0D146A00FA146003753200C3E53298401D8E
:10147700120FDD120546153275310078998673C251
:10148700AF120584D2AF7898867312055A120550A9
:10149700E52A7005307402411E780120740278062F
:1014A700C3E55C9840A112055AE52A700302121E93
:1014B700C2AF120FDDE4F522F523F524F525F52655
:1014C700F567D2AF7885E6C333F565E4F544F545AE
:1014D700F546F547F548F570F52CF52DF537757098
:1014E7000875BB1E12054612092F30EDFDA8BDA9D0
:1014F700BEE97001F8887112093375700875BB1E53
:10150700115EC2AF7561FF1209EC85226185226207
:10151700852263D2AF7522017524017525017526D1
:1015270001856069756A017888E6B40307C27D3072
:101537007602D27DD268D269753300120F36120F48
:1015470065120A0C120A13120A0C120A13120A0C59
:10155700120C93120665120D91120DD8120A13126E
:101567000C82306E03120705206603120858306696
:1015770003120888120D91120E0D120A13120C9302
:10158700306E03120741120D91120E84120A1312C4
:101597000C82306E0312079F120D91120EB3120ABE
:1015A70013120C93306E031207FC120D91120F36B3
:1015B700120A1312092F120C82120D91120F6512C3
:1015C7000933120A1330692C85646185646285606A
:1015D70069756A0179187A0CC3E533994009C269BC
:1015E700D26A8A350215FBC3E55C940140030215F4
:1015F70057021666306A25206C22E535147006C23C
:101607006AD26BA157F535C3E55C94014003021517
:10161700577888E6C394036003021666753600C3DD
:10162700E55F94014009856462856069756A0178A0
:10163700FA79A4E760027803C3E55F985021307414
:1016470004E52A601A78F0306C058564617820C358
:10165700E541985002A1570536E55C6002C16975FE
:101667003600C2AF120FDD7887E6FE7602115E788C
:1016770087EEF6E4F522F523F524F525F526F5653D
:10168700752C00752D00D2AF12055A120FDD78A404
:10169700E66006D293D295D297307406E52A700297
:1016A700411E788DE6C39401400261018149901A79
:1016B7000D7820121745E520B4A50CA3121745E5B0
:1016C70020B45A030216E3757CA5757DF1120FF25B
:1016D700121703757C00757D00021702901A0378B4
:1016E700807B0A121745A308DBF9901A0F788C7BC9
:1016F70019121745A308DBF9901A2822C2AF12174F
:1017070088121765901A00740E12174AA3740912EB
:10171700174AA3741512174A901A0378807B0A1286
:101727001749A308DBF9901A0F788C7B1912174910
:10173700A308DBF912179B121779901A2822E49352
:10174700F622E6438F01538FFDFFC3E583941C40C8
:101757000122EF857CB7857DB7F0538FFE22438F3B
:1017670002438F01857CB7857DB7901A0DF0538FA3
:10177700FC22901A0D74A5F14A901A0E745AF14A78
:10178700227A3079D07820901A40F145E520F70980
:10179700A3DAF7227A3079D0901A40E7F14A09A301
:1017A700DAF922AB74A875BB01027980BB02027912
:1017B70081BB03027982BB04027994BB050279835A
:1017C700BB06027986BB07027992BB08027987BB01
:1017D7000902799CBB0A027988BB0B027989E8F771
:1017E700227C0512055FDCFB22C2AF12056F1205D2
:1017F7007612057D12058412055012056F120576C3
:1018070012057D12058412055012056F1205761216
:10181700057D120584D2AF22C2AF12058412057D61
:1018270012057612056F12055012058412057D12F6
:10183700057612056F12055012058412057D1205F3
:101847007612056FD2AF22AE74AF75C2AF12056FB5
:1018570012056F12056F120550DEF212058412058C
:0F18670050DFF8D2AF221217F01217E81217E86D
:10187600757401757501757600114E7C05AD5C12A7
:10188600055FC3ED955C70F5C3E55C9401400AC342
:10189600E55C94FF40370218B01217AA121703121C
:1018A60017F0C2AF75EF161217E8DCD10576C3E55F
:1018B600769403500280C21217E80575E5741490F9
:1018C600009F93F808C3E57598500280A91217E89F
:1018D6001217E80574C3E574940C50028095120F34
:0C18E600F2121703C2AF75EF161217E8DC
:0319FD000211656F
:101A00000E091507070104FFFF07020101A55A018E
:101A100000B4FFFFFF03FF01FF25D078C804FF01DA
:091A200000FF10010100FF00FFAE
:101A4000235467794B4631323041485623202020B9
:101A500023424C48454C4923463331302320202033
:101A60002020202020202020202020202020202076
:101C0000C2AFC2D353D9BF7581C043B20343FF8073
:101C1000752438752503B1DC7529A5752AF175E29F
:101C20004043F10853A4F775D4FFD2837DFA7803BB
:101C300079E67C10752200752300901DE97B0675FE
:101C400024987525013083028145208308D8FBD96B
:101C5000F9DCF781B7308308D8FBD9F9DCF781B715
:101C6000B19CE493A3C39A6004DDC381B7DBDBB10D
:101C70008E6002812E7B08E493FAA3B16FDBF87AC1
:101C800030B16F752200752300B18EEAFCEBFDC305
:101C9000ED94FE400EB18E8A278B28ED30E0048A49
:101CA000828B83B18E7AC270D8C3ED94FE601950D6
:101CB000CEBD002BEC600F7520007521FF7529004B
:101CC000752A000200008100A827A9280809D80465
:101CD000D90281DCB192EA89AAF281CE0D81A3C337
:101CE000ED94035053EDA2E092007AC5C3E58294CF
:101CF00000E583941C508A200010438F02438F011B
:101D00008529B7852AB7F0300029A827A92808090E
:101D1000438F01538FFDD804D902A133C3E58394C7
:101D20001C4003A3A11689AAE28529B7852AB7F02A
:101D3000A3A116538FFC817F7AC1BD030CE493A34A
:101D4000FAB153DCF8B14B817F8181AA22AB23B178
:101D50006FEBFAEA6222752608C3E52313F523E543
:101D60002213F52250066323A0632201D526EAB18F
:101D7000DCB1DC75260AEAF4200102D283300102CC
:101D8000C283B1DCC3134002C201D526EB22B1925B
:101D9000EAFB208302A192308302A197752608AE48
:101DA00024AF25C3EF13FFEE13FEB1E0B1DCC3EAAD
:101DB000133083024480FA30E703632201C3E52332
:101DC00013F523E52213F52250066323A0632201B5
:101DD000D526D9E52265236523F52222AE24AF2539
:101DE0000E0FDEFEDFFCD20122424C48656C6934E6
:071DF000373164F310060116
:00000001FF
